:0614000002148B024A7D7C
:01140B0032AE
:0114130032A6
:01141B00329E
:011423003296
:01142B00328E
:031433000242F181
:01143B00327E
:011443003276
:03144B000251B596
:03145300021AC0BA
:03145B00021D9AD5
:011463003256
:03146B00024374C5
:011473003246
:01147B00323E
:03148300024DA176
:0314E90002148664
:03148600022E54DF
:1014EC00AF83E58290F554F0EFA3F0C2A0C2A4D272
:1014FC00A375E10490DF3BE0FFBF01F890F554E0E9
:10150C00FEA3E090DF06EEF0C2A090FCACE024FF5E
:10151C0092A4E06401FF24FF92A375E10290DF3BEB
:10152C00E0FFBF0DF8227E007F0090FC48E0FCA39A
:10153C00E0FD8E028F03C3EA9CEB9D503AEE240033
:10154C00FCEF34F0FD90FC46E0F514A3E0F5158AB1
:10155C00828B83C007C006C005C0041256EAAA825B
:10156C00AB83D004D005D006D0078C828D83EAF0F3
:10157C000EBE00B60F80B322E58290F556F0E0FF68
:10158C00E59CC39FF59CE59C24FAF59C439E10D2E8
:10159C00BA22AF9E74EF5FF59E22AF83E58290F581
:1015AC005AF0EFA3F090FC41E060139058AC12435A
:1015BC00E390FC41E0F5821244257582EF2290FC09
:1015CC00417406F090DF3BE0FFBF130280F6C2913E
:1015DC0090F557E0FEA3E0FF90FCA8EEF0EFA3F02F
:1015EC0090FCA274F1F0E4A3F090FC387472F074E7
:1015FC00F3A3F090FCA0E4F0A3F090FC53F090FC6B
:10160C009CF090FC52F090FC9E04F0E4A3F090FC53
:10161C009D7402F090F55CE4F090000012175F905E
:10162C00F55AE0FEA3E0FF90F559E0FD7B007C004D
:10163C008D017A00C3EB99EC9A50548B02EA75F049
:10164C00F0A42EF9E43FFA90F55C74F0F089828AEC
:10165C0083C007C006C005C004C00312175FAA826E
:10166C00D003D004D005D006D007EA601B9058FEFA
:10167C00C0021243E3D00290FC41E4F08A82C00223
:10168C00124425D0028A82220BBB00A40C80A190AC
:10169C00FCABE0FF30E33390FCA8E0FEA3E0FFEEF0
:1016AC00540F602690FCA8E0FEA3E053060F7F00C9
:1016BC007410C39EFEE49FFF90FCA8E0FCA3E0FD29
:1016CC0090FCA8EE2CF0EF3DA3F090FCA8E0FEA35C
:1016DC00E0FFC374FF9EE49F502390FCA8E0FEA3A0
:1016EC00E090DF02EEF090DF04E0FF74FC5FF0E0CE
:1016FC00FF74024FF090FCAA7401F0801290FCA8C9
:10170C00E0FEA3E0FF90DF02EEF090FCAAE4F09084
:10171C00FCACE024FF92A0C2A490FCACE0640124D9
:10172C00FF92A375E1037E607FEA90DF3BE0FDBD95
:10173C00130280091EBEFF011FEE4F70EDD291EE19
:10174C004F700C90FC667413F09059161243E375AD
:10175C00820022AF83E58290F55DF0EFA3F090F567
:10176C005CE0FF240F500A9059271243E37582FF67
:10177C0022EF703E90FC52E4F090FC52E0FE90FCA4
:10178C009DE0FDC3EE9D502190FC52E075F0F1A45C
:10179C002472F58274F335F0F583E4F090FC52E09A
:1017AC00FE0E90FC52EEF080D090FC52E4F075826C
:1017BC00002290FC41E0FE601DBE061E90FC52E033
:1017CC00601890DF3BE0FEBE1302800E90FC41746B
:1017DC0007F07582ED227582ED2290FC52E075F0D7
:1017EC00F1A42472FD74F335F0FE8D828E83E060DB
:1017FC000A90FC667418F07582FE228D828E8374BA
:10180C00FFF090FC52E075F0F1A42472FD74F335F6
:10181C00F0FE0DBD00010E7C0090F55DE0FAA3E03A
:10182C00FB8A148B158C168F037F008B178F188DEA
:10183C00828E838CF0C007C003125611D003D007E0
:10184C0090FCABE0FE20E30302190790FC52E0751C
:10185C00F0F1A42472FD74F335F0FE0DBD00010E01
:10186C0090FC7DEBF0EFA3F08D828E8312532FAEA4
:10187C008290F55CEEF090FCABE0FF530704BF04E4
:10188C003F90FC52E075F0F1A42472FD74F335F036
:10189C00FF0DBD00010F8E037C0090FCABE0FA53F2
:1018AC0002F090FC81EDF0EFA3F090FC83EBF0ECF8
:1018BC00A3F090FC85EAF08D828F83125369803BF4
:1018CC0090FC52E075F0F1A42472FD74F335F0FF36
:1018DC000DBD00010F7C0090FCABE0FB5303F090BE
:1018EC00FC88EDF0EFA3F090FC8AEEF0ECA3F09006
:1018FC00FC8CEBF08D828F831253B290FC52E0750E
:10190C00F0F1A42472FE74F335F0FF90F55CE0FD69
:10191C008E828F83F090FC52E0FF0F90FC52EFF020
:10192C0090FC9DE0FEEFB5060590FC52E4F075824C
:10193C000022AF83E58290F55FF0EFA3F090FC41BD
:10194C00E0FF6014BF0102800F9059411243E390F5
:10195C00FC41E0F58212442512159E90FC4AE4F0FD
:10196C00A3F090FC4AE0FEA3E0FF8E828F83121A54
:10197C004090DF3BE0FFBF0DF890DF3AE0FF5307EC
:10198C007FBF6000402790FC4AE0FEA3E0FF0EBE44
:10199C0000010F90FC4AEEF0EFA3F0D29190000AF8
:1019AC00125028C29190000A12502880B590FC4128
:1019BC007402F090FC67E0FCA3E0FDA3E0A3E090D0
:1019CC00FC4CECF0EDA3F090F55FE0FEA3E0FF9093
:1019DC00FC50EEF0EFA3F02290FC41E4F090FC6799
:1019EC00E0FCA3E0FDA3E0A3E090FC4CECF0EDA345
:1019FC00F02290FC417404F090FC67E0FCA3E0FD45
:101A0C00A3E0A3E090FC4CECF0EDA3F02290FC41A1
:101A1C007405F090FC54E4F0A3F090FC67E0FCA398
:101A2C00E0FDA3E0A3E090FC4CECF0EDA3F075829C
:101A3C0000021584AF83E58290F561F0EFA3F0907E
:101A4C00F561E0FEA3E0FFEE2400F582EF34F0F543
:101A5C0083E0FF7E008F828E830214ECAF83E582DD
:101A6C0090F563F0EFA3F090F563E0FEA3E0FF9038
:101A7C00F370EEF0EFA3F0222290FC4AE0FEA3E01C
:101A8C00FF0EBE00010F90FC4AEEF0EFA3F0C3EE88
:101A9C009470EF9403400790FC4AE4F0A3F090FCA0
:101AAC004AE0FEA3E0FFEE2400F582EF34F0F5836C
:101ABC00E0F58222C021C0E0C0F0C082C083C00724
:101ACC00C006C005C004C003C002C001C000C0D025
:101ADC0075D00090FC3DE02401F0A3E03400F090C0
:101AEC00FC42E0FEA3E0FF90FC3DE0FCA3E0FDEC3B
:101AFC00B5060BEDB5070790FC3DE4F0A3F090FCA8
:101B0C003DE0FEA3E0FFBE0005BF0002800BBE015E
:101B1C0005BF00028068021C8290FC3DE0FEA3E041
:101B2C008E077E00AC9C7D00EC4206ED420790FCDB
:101B3C004EEEF0EFA3F090FC4AE0FEA3E0FF0EBEE9
:101B4C0000010F90FC4AEEF0EFA3F090FC48E0FC93
:101B5C00A3E0FDC3EE9CEF9D400790FC4AE4F0A38C
:101B6C00F090DF3BE0FFBF1303021D7D90FC4AE0C9
:101B7C00FEA3E0FF8E828F83121A40021D7D90FC23
:101B8C0041E0FFBF05028003021D7D900019125039
:101B9C002890F567741CF090FC4AE0FEA3E090F5E9
:101BAC0068EEF090FC4AE0A3E090F569F090F56ADD
:101BBC007442F090F56B744CF090F56C7441F090AD
:101BCC00F56D7448F090F56E7442F090F56F744CAE
:101BDC00F090F5707441F090F5717448F090F572D6
:101BEC007442F090F573744CF090F5747441F0906D
:101BFC00F5757448F090F5767442F090F577744C66
:101C0C00F090F5787441F090F5797448F090F57A8D
:101C1C007442F090F57B744CF090F57C7441F0902C
:101C2C00F57D7448F090F57E7442F090F57F744C1D
:101C3C00F090F5807441F090F5817448F090F58245
:101C4C007420F090FC56741CF0E4A3F090FC58F057
:101C5C00A3F090FC5AF0A3F090F5681246D090FCDB
:101C6C0054E0FEA3E0FF0EBE00010F90FC54EEF01A
:101C7C00EFA3F0021D7D90FC41E0FFBF03028065E5
:101C8C00BF04028008BF05028003021D7D90FC4C3E
:101C9C00E0FEA3E0FF90FC67E0FAA3E0FBA3E0FC0E
:101CAC00A3E0FD8E008F01E4FEFFEAC398FAEB99E6
:101CBC00FBEC9EFCED9FFDC374649AE49BE49CE4F6
:101CCC009D502290596F1243E390FC417405F090A3
:101CDC00FC67E0FCA3E0FDA3E0FEA3E0FF90FC4C5E
:101CEC00ECF0EDA3F090FC53E075F0F1A42472FE3F
:101CFC0074F335F0FF8E828F83E0607590001912BB
:101D0C00502890FC53E075F0F1A42472FE74F33566
:101D1C00F0FF90DF04E05401FDB40100E4332EFD2C
:101D2C00E43FFC8E828F83E090FC56F0E4A3F090AD
:101D3C00FC58F0A3F090FC5AF0A3F08D828C831227
:101D4C0046D090FC53E075F0F1A42472F58274F344
:101D5C0035F0F583E4F090FC53E0FF0F90FC53EF6B
:101D6C00F0BF0200400590FC53E4F090598D1243F3
:101D7C00E3D0D0D000D001D002D003D004D005D015
:101D8C0006D007D083D082D0F0D0E0D02132329070
:101D9C00FC41E4F090FC52F090FC53F090FC4AF0C3
:101DAC00A3F090FC467453F0E4A3F090FC487453F9
:101DBC00F0E4A3F090FC4EF0A3F090FC4CF0A3F0F8
:101DCC0090FC427406F0E4A3F090FC44F0A3F09075
:101DDC00FC50F0A3F090FC54F0A3F012153290FCE0
:101DEC0041E4F0759DDC859E9E439E0443CB1022FE
:101DFC00021D9B90224712339C90FC67E4F0A3F0E9
:101E0C00A3F0A3F0121DFC90F583E4F090F584741C
:101E1C0032F074F8A3F02290FC41E0FFBF00030203
:101E2C00217CBF010302204DBF0203021F4BBF03E5
:101E3C000302217CBF040302217CBF050302215D48
:101E4C00BF060122BF40028006BF4102804822C269
:101E5C00A0C2A4D2A375E10490DF3BE0FFBF01F860
:101E6C0090DF0374E5F090DF047404F090DF0774E6
:101E7C0012F090DF08E4F090DF147410F090DF178C
:101E8C00E0FF74C04FF090FC417441F090F5847405
:101E9C0032F074F8A3F090F583E4F090FC54E0FE7B
:101EAC00A3E0FF90F583E0FDFB7C00C3EB9EEC9F71
:101EBC00505D90DF06EDF0C2A0C2A4D2A375E10480
:101ECC0090DF3BE0FFBF01F8C2A090FCACE024FF28
:101EDC0092A4E06401FF24FF92A375E10290DF3B22
:101EEC00E0FFBF0DF890000212502890F584E0FE40
:101EFC00A3E0FF90F583E02EFEE43FFF90DF3AE095
:101F0C00FD8E828F83F090F583E02401F0808CC2EB
:101F1C00A0C2A4D2A375E10490DF3BE0FFBF01F89F
:101F2C0090FC54E0FEA3E08E3375340090F584E011
:101F3C00F535A3E0F536753201758243022E86E540
:101F4C000F700302203B90FC65740DF0AF9A74FE89
:101F5C005FF59AE50F20E40302203B90FC417403EB
:101F6C00F090FC3FE0FEA3E08E8212158490599B0A
:101F7C001243E390FC3FE0FEA3E0FF8E828F8312BE
:101F8C00444090F831E025E0FEE42432FFEE34F8D2
:101F9C00FE8F828E831243E390F831E0FFB4010090
:101FAC00E433FF90F583F0EF2436FDE434FCFE8D32
:101FBC00828E83E0707290DF04E0FE30E0378F0693
:101FCC00EE2EFDE42432F582ED34F8F583E0FE8E3E
:101FDC00337534008F06EE2EFDE42432FEED34F81A
:101FEC00FD74012EF535E43DF536753201758242EE
:101FFC00122E86802290DF02E0FE8E33E4F534EF61
:10200C002FFEE42432FFEE34F8FE8F358E36753217
:10201C0001758242122E8690F583E0FF2436F582FC
:10202C00E434FCF5837401F0AF0F74EF5FF50FD25D
:10203C000010AF02C200750F00A20092AF439A01CC
:10204C0022E50F700302214B90FC65740DF0AF9AE2
:10205C0074FE5FF59AE50F20E40302214B90F831F2
:10206C00E0FF90F583B40100E433F09059B01243D3
:10207C00E390F583E025E0FEE42432FFEE34F8FE35
:10208C008F828E8312444090F583E025E0FEE42499
:10209C0032FFEE34F8FE8F828E831243E390F831D8
:1020AC00E0FFB40100E433FF90F583F0EF2436FD3C
:1020BC00E434FCFE8D828E83E0707290DF04E0FECF
:1020CC0030E0378F06EE2EFDE42432F582ED34F845
:1020DC00F583E0FE8E337534008F06EE2EFDE4247E
:1020EC0032FEED34F8FD74012EF535E43DF5367510
:1020FC003201758242122E86802290DF02E0FE8E23
:10210C0033E4F534EF2FFEE42432FFEE34F8FE8F87
:10211C00358E36753201758242122E8690F583E02B
:10212C00FF2436F582E434FCF5837401F0D2001000
:10213C00AF02C200AF0F74EF5FF50FA20092AFD2E7
:10214C000010AF02C200750F00A20092AF439A01BB
:10215C002290FC54E0FEA3E0FF90FC48E0FCA3E0DE
:10216C00FDC3EE9CEF9D50012290FC417404F022C3
:10217C00E50F70012290FC65740DF0E50F54307082
:10218C00012290F831E0FFB40100E433FF90F583B5
:10219C00F0EF2436FDE434FCFE8D828E83E0600388
:1021AC0002223490DF04E0FE30E0378F06EE2EFD85
:1021BC00E42432F582ED34F8F583E0FE8E33753489
:1021CC00008F06EE2EFDE42432FEED34F8FD740192
:1021DC002EF535E43DF536753201758242122E86A8
:1021EC00803590FC97E0E0600A90FC9AE0FDA3E05B
:1021FC00FE800890DF02E0FCFD7E00EF2FFCE42463
:10220C0032FFEC34F8FC8F358C367532018D338E01
:10221C0034758242122E8690F583E0FF2436F582C7
:10222C00E434FCF5837401F0D20010AF02C200AFAD
:10223C000F74CF5FF50FA20092AF2290F7E3E0FD91
:10224C00A3E0FEA3E0FF90F7E8E0FCBC42028003B1
:10225C00022BE290F7E9E0FC24BE5003022BD4ECF5
:10226C00240A83F582EC244683F583E473D4D44D9D
:10227C0095D400BBD9EC255E82C563D4D429A8CFF4
:10228C0042677AE65A8FD4D4D4D4D4D4D439C20980
:10229C00FF22D4D4D4D4D4D4D4D4D4D4D4D4D4D479
:1022AC00D4D4D4D4D4D4D4D4D4D4D4D4D4FD372BFF
:1022BC002B23252B2424242425252525262B2B29AB
:1022CC0029292A2A2A2A28292B2B2B2B2B2B2B2B5F
:1022DC002B2B292A2B2B2B2B2B2B2B2B2B2B2B2B45
:1022EC002B2B2B2B2B2B2B2B2B2B2B2B2B2B2B223B
:1022FC0023C007C006C00512159ED005D006D00716
:10230C0090FC417440F08D828E838FF0125849FC02
:10231C007B0090FC54ECF0EBA3F090F809EDF0EEA0
:10232C00A3F0758201124135022BE290FC41E4F0DE
:10233C0090F809EDF0EEA3F0758201124135022BF5
:10234C00E290FC41E060099059CA1243E3022BE28F
:10235C008D828E838FF0125849FC7B0090F586ECB1
:10236C00F0EBA3F08D828E83A3E0FAE4F92CFCEA67
:10237C003BFB90F586ECF0EBA3F08D828E83A3A350
:10238C00A3A3E0FA8A0889098D828E83A3A3A3A351
:10239C00A3E0FAE42508F508EA3509F50990FC3ABA
:1023AC00E4F0A3F074062DF9E43EFA90FC56ECF040
:1023BC00EBA3F090FC58E4F0A3F090FC5AE508F085
:1023CC00E509A3F089828A83C007C006C0051246BE
:1023DC00D0AC82D005D006D0078D828E838FF0ECE6
:1023EC001256B290F809EDF0EEA3F075820112418D
:1023FC0035022BE28D828E838FF012584990FC9A15
:10240C00F0E4A3F08D828E83A3E0FB7C0090FC9A19
:10241C00E0F9A3E0FA90FC9AEC29F0EB3AA3F090E7
:10242C00FC9AE0A3E090FC9AE0F5F0A3E045F060A4
:10243C004B90FC977401F090FC98E0A3E090FC9812
:10244C00E0F5F0A3E045F070471245FD90FC9AE0F2
:10245C00FBA3E0FC90FC98EBF0ECA3F090FC98E074
:10246C00FBA3E090DF02EBF090DF04E0FC74FC5C7B
:10247C00F0E0FC74024CF012459D801490FC97E443
:10248C00F090FC98F0A3F090FC9AF0A3F01245FDAC
:10249C0090F7E8E0FC90F7E9E0F53275359A75367F
:1024AC00FC7533017534008C82122E86022BE28D62
:1024BC00828E838FF012584990FCABF090F809EDA6
:1024CC00F0EEA3F0758201124135022BE290F8096F
:1024DC0074ABF074FCA3F0758201124135022BE24F
:1024EC0090FCABE0FC5304F090FC797406F090FC8B
:1024FC007AECF08D828E838FF0C007C006C0051277
:10250C0052D7D005D006D00790F809EDF0EEA3F025
:10251C00758210124135022BE290FCABE0FC5304A7
:10252C00F090FC797404F090FC7AECF08D828E8340
:10253C008FF0C007C006C0051252D7D005D006D008
:10254C000790F809EDF0EEA3F075821012413502F8
:10255C002BE28D828E838FF012584990FCACF0E008
:10256C00FC74015CF090F809EDF0EEA3F0758201BB
:10257C00124135022BE290F80974ACF074FCA3F014
:10258C00758201124135022BE28D828E838FF012FF
:10259C005849FC7B008C828B83C007C006C0051297
:1025AC001A68D005D006D00790F809EDF0EEA3F02C
:1025BC00758201124135022BE290FC41E0601C8DCA
:1025CC00828E838FF074EF1256B290F809EDF0EE14
:1025DC00A3F0758201124135022BE28D828E838F1E
:1025EC00F0125849FC7B0090F586ECF0EBA3F08DD3
:1025FC00828E83A3E0FAE42CFCEA3BFB90F586EC9C
:10260C00F0EBA3F08D828E83A3A3E0FA90FC3AE466
:10261C00F0A3F074032DF8E43EF990F557ECF0EBD1
:10262C00A3F090F559EAF088828983C007C006C0F0
:10263C00051215A6AC82D005D006D0078D828E83EC
:10264C008FF0EC1256B290F809EDF0EEA3F0758213
:10265C0001124135022BE28D828E838FF012584984
:10266C00FB7C0090F586EBF0ECA3F0EB4C600302E6
:10267C00276B90FCA8E0A3E090FCA8E0F5F0A3E0A9
:10268C0045F0601C90DF3BE0FABA1314900028C0B0
:10269C0007C006C005125028D005D006D00780D23E
:1026AC0090FCA8E0A3E090FCA8E0F5F0A3E045F0D6
:1026BC00606B9059EFC007C006C0051243E390FC55
:1026CC00A8E0F9A3E0FA89828A8312444090F3725D
:1026DC00E0F58212442590F463E0F582124425D093
:1026EC0005D006D00790FC667412F08D828E838F15
:1026FC00F074EC1256B2C291C007C006C005124568
:10270C0078D005D006D00790FC41E4F090F809EDA4
:10271C00F0EEA3F0758201124135022BE2C29190CA
:10272C00FC41E4F08D828E838FF01256B2905A03E6
:10273C00C007C006C0051243E390FC3AE0F9A3E0E1
:10274C00FA89828A83124440D005D006D00790F8CB
:10275C0009EDF0EEA3F0758201124135022BE290E7
:10276C00FC41E0FABA06028061905A13C007C00619
:10277C00C0051243E3D005D006D00790FC66E0FA02
:10278C00BA121B8D828E838FF074EC1256B290F8B5
:10279C0009EDF0EEA3F0758201124135801F90FC1B
:1027AC00667417F08D828E838FF074EF1256B29090
:1027BC00F809EDF0EEA3F0758201124135C29112C9
:1027CC00457890FC41E4F0022BE274012DF9E43ED3
:1027DC00FA90F55CEBF089828A83C007C006C005CD
:1027EC0012175FAC82D005D006D0078D828E838FF6
:1027FC00F0EC1256B28D828E838FF0125849FBEC9E
:10280C00603BBBFE028036905A1CC007C006C00558
:10281C001243E3D005D006D0078D828E838FF01241
:10282C005849F582C007C006C005124425C2911252
:10283C004578D005D006D00790FC41E4F090F8091B
:10284C00EDF0EEA3F0758201124135022BE28D8280
:10285C008E838FF0125849FB7C0090F586EBF0ECE0
:10286C00A3F0C374F09BE49C50199059271243E3D6
:10287C0090F8097486F074F5A3F075820112413555
:10288C00022BE290FC52E075F0F1A42472F974F37F
:10289C0035F0FA89828A83E06019905A291243E351
:1028AC0090F8097486F074F5A3F075820112413525
:1028BC00022BE28B0089828A83E8F090FC52E0754F
:1028CC00F0F1A42472F974F335F0FA09B900010A95
:1028DC00890A8A0B750C0074012DF9E43EFA8914EF
:1028EC008A157516008B178C18850A82850B8385C3
:1028FC000CF012561190FC52E0FC0C90FC52ECF0D7
:10290C00BC0200400590FC52E4F090F8097486F08B
:10291C0074F5A3F0758201124135022BE28D828E83
:10292C00838FF0125849FC7B0090FC46ECF0EBA333
:10293C00F090FC46E0F9A3E0FAC374709C74039B1E
:10294C00402E74022DFBE43EFC8B148C1575160086
:10295C0089178A1890F00075F00012561190F8093A
:10296C007446F074FCA3F0758202124135022BE21E
:10297C0090F809744AF0745AA3F075820812413524
:10298C00022BE290FC46E0FBA3E090F8097400F007
:10299C0074F0A3F08B82124135022BE2121A857B64
:1029AC00008B83121A4090FC4AE0FBA3E0FC90F8E9
:1029BC0009EB2400F0EC34F0A3F0758201124135E0
:1029CC00022BE28D828E838FF0125849FC7B008C97
:1029DC00828B83C007C006C0051214ECD005D0064C
:1029EC00D00790F809EDF0EEA3F075820112413595
:1029FC00022BE2758200C007C006C005121584D0F8
:102A0C0005D006D00790F809EDF0EEA3F075820121
:102A1C00124135022BE2C007C006C00512159ED02C
:102A2C0005D006D00790F809EDF0EEA3F075820101
:102A3C00124135022BE28D828E838FF0125849FCA5
:102A4C007B0090FC42ECF0EBA3F090F809EDF0EE7B
:102A5C00A3F0758201124135022BE290F809744201
:102A6C00F074FCA3F0758204124135022BE28D82C6
:102A7C008E838FF0C007C006C0051243A2D005D0CC
:102A8C0006D0078D828E838FF0125849F582C007CD
:102A9C00C006C005124425D005D006D0078D828E05
:102AAC00838FF0125849FC7B008C148B158B167598
:102ABC0017158B1890FC4175F000C007C006C005B7
:102ACC00125611D005D006D00790F809EDF0EEA300
:102ADC00F0758215124135022BE290FC3DE0FBA310
:102AEC00E0FC90FC44EBF0ECA3F090F8097441F09E
:102AFC0074FCA3F0758215124135022BE28D828E87
:102B0C00838FF0125849FC7B008C828B83C007C0EA
:102B1C0006C00512193ED005D006D00790F809ED75
:102B2C00F0EEA3F0758201124135022BE290FC67A6
:102B3C00E0F9A3E0FAA3E0A3E090FC4CE9F0EAA3EF
:102B4C00F08D828E838FF0125849FC90FC41F090EE
:102B5C00FC41E0FBEC24FA404DEB2B2B902B6C73DF
:102B6C00022B7E022B7E022B7E022BA0022BA002BC
:102B7C002B8FC007C006C00512159ED005D006D0FD
:102B8C00078023C007C006C005121A19D005D0064D
:102B9C00D0078012758200C007C006C005121584CC
:102BAC00D005D006D00790F809EDF0EEA3F07582B1
:102BBC0001124135802090F8097441F074FCA3F0A7
:102BCC00758201124135800E90F809EDF0EEA3F0FC
:102BDC00758201124135900000222290F7F1E0FF3E
:102BEC00BF013990F7D1E0FEA3E0FF90F7F4E0FCD1
:102BFC00A3E0FD90F7D4E0FAA3E0FBEA4B601D8E56
:102C0C00828F83E0F9A3AE82AF838C828D83E9F04F
:102C1C00A3AC82AD831ABAFF011B80DF90F7DAE018
:102C2C0054FDF090DE11E0FF74084FF022AE82AF3D
:102C3C0083E0FD20E703022D328E828F83A3E0FD1B
:102C4C00601DBD0102802ABD0202803BBD030280D3
:102C5C005ABD04028076BDFE03022CF4022D32759F
:102C6C00370275380090FC6575F000123134022D76
:102C7C003290DE00E0FD7C007539288C3A8D828C18
:102C8C00831231A8022D328E828F83A3A3E0FCA382
:102C9C00E0FD74062EF582E43FF583E0F539A3E000
:102CAC00F53A8C828D831231A8807B8E048F057B44
:102CBC000074062EF582E43FF583E0F537A3E0F5CA
:102CCC00388C828D838BF0123134805A90F7D1E09E
:102CDC00FBA3E0FCA3E0FD753910753A008B828CE8
:102CEC00838DF01231A8803E74022EFEE43FFF7DEE
:102CFC0000756B52756C5A756D807514048D158E3C
:102D0C00828F838DF01250F4E5828583F045F0605C
:102D1C0012D29190012C125028C29190012C125079
:102D2C0028800375C9839000002290DF2FE4F09077
:102D3C00DF30F090DF31F090DF00740CF090DF01A9
:102D4C00744EF090DF0274FFF090DF037440F0904B
:102D5C00DF04E4F090DF05F090DF06F090DF0774FD
:102D6C0006F090DF08E4F090DF097424F090DF0A9D
:102D7C00743AF090DF0B74F1F090DF0C74CAF090A1
:102D8C00DF0D74A3F090DF0E7401F090DF0F74234D
:102D9C00F090DF107411F090DF117436F090DF12A8
:102DAC007407F090DF13740FF090DF147418F09028
:102DBC00DF1514F090DF16746CF090DF177403F0CD
:102DCC0090DF187440F090DF197491F090DF1A7452
:102DDC0056F090DF1B7410F090DF1C74E9F090DF5C
:102DEC001D742AF090DF1EE4F090DF1F741FF0902A
:102DFC00DF237488F090DF247431F090DF257409A0
:102E0C00F090DF2E74C0F090DF07C4F090DF0974EF
:102E1C0025F090DF0A7495F090DF0B7455F090DF7D
:102E2C001A74B6F090DF1B7410F090DF1C74EAF08B
:102E3C0090DF1D742AF090DF1EE4F090DF1F741FEA
:102E4C00F0221251760251A2122E4E12448A1251C5
:102E5C00DC1230FF12463C121DFF12312ED2AF1283
:102E6C002FD1D291900002125028C29190000A12D8
:0A2E7C005028124166121E2380F850
:1058AC0043616E6E6F742063616C6C207472616EF8
:1058BC00736D69745F6C6F6E67207768696C6520B7
:1058CC004648535320486F7070696E67206F722082
:1058DC00616C72656164792070726F636573736952
:1058EC006E67207472616E736D69745F6C6F6E6736
:1058FC0021004D41435F74782829207265747572BC
:10590C006E6564206572726F72006E6576657220CA
:10591C00656E74657265642054580046485353781C
:10592C006D6974206D65737361676520746F6F208A
:10593C006C6F6E6700464853532073746174652016
:10594C00656E746572696E672053594E4348494EB3
:10595C00472066726F6D2077726F6E67207374616B
:10596C0074650053594E43485F4D41535445522082
:10597C002D3E2053594E43494E474D4153544552A9
:10598C000046485353786D697420646F6E65006EE1
:10599C006574776F726B207061636B6574287379B3
:1059AC006E6329006E6574776F726B207061636B28
:1059BC00657428646973636F766572792900637204
:1059CC0061702C20706C6561736520757365204661
:1059DC00485353786D6974282920696E7374656116
:1059EC0064210064726F706F75742066696E616CEF
:1059FC0020776169742100746F74616C2062797412
:105A0C0065732074783A00756E64657272756E00F9
:105A1C00627566666572206572726F720073746966
:105A2C006C6C2077616974696E67206F6E20746886
:105A3C0065206C617374207061636B6574004E4FEC
:0B5A4C00204445414C005253544E00D2
:102E8600AF827E0190DE0E7405F090FC657412F040
:102E9600E53345347003022FC77C107D2790DE1181
:102EA600E0FB30E00D90FC667401F01CBCFF011DD8
:102EB60080EBEC4D7014D2919003E8125028C29129
:102EC6009003E812502890FFFF22BE012C7E00904E
:102ED600DE2A7440F0EFF0E532F0AC337D00ECF022
:102EE600E534F0C3743B9533E4953450067C3B7D62
:102EF60000801AAC33AD348014C374409533E49526
:102F06003450067C407D008004AC33AD347480259B
:102F16002942D6852682852783AA35AB368B01E9D9
:102F2600F0852682852783A3EAF085268285278376
:102F3600A3A374DEF0852682852783A3A3A3742A20
:102F4600F0852682852783A3A3A3A3A3ECFBF085A4
:102F56002682852783A3A3A3A3E054E0F0852682D7
:102F6600852783A3A3A3A3A3A3A3E0543F4440F0D0
:102F7600852682852783A3A3A3A3A3A3A3E054CF77
:102F8600F0E52942D6E52942D7E52955D160FAE58B
:102F960029F452D190DE0E7405F090DE11E0FB7438
:102FA600014BF0E533C39CF533E5349DF534EC2550
:102FB60035F535ED3536F53690FC657413F0022E91
:102FC6009690FC657414F090000022E522700512BC
:102FD600416680F722AFBE747F5FF5BE43BE809028
:102FE600DE0B7407F090DE077411F090DE0914F022
:102FF600438C10AF8C74FE5FF58CD2BD439A02757C
:103006008900C2C5758B00C2E843A90243B902858F
:103016002682852783A3A3A3A3E054E0F085268216
:10302600852783A3A3A3A3A3A3E0549F4420F085ED
:103036002682852783A3A3A3A3A3A3A3E04408F022
:10304600852682852783A3A3A3A3A3A3A3E054FC79
:103056004401F090DE01E0FF74FE5FF0E4F525F533
:1030660023F524F52290DE0EF090DE107408F09021
:10307600DE13F090F7DBE4F090F7DAF090F7CFF09C
:10308600A3F090F7D17488F074F5A3F0E4A3F09060
:10309600F7D4F0A3F090F7D6F090F7D7F090F7D8E2
:1030A600F0A3F090DE0E7405F090DE107408F09038
:1030B600DE13F090DE12E0FF74014FF090DE15E0B3
:1030C600FF74014FF090F7EDE4F090F7ECF090F715
:1030D600E1F0A3F090F7E374C8F074F5A3F0E4A36D
:1030E600F090F7E6F0A3F090F7E8F090F7E9F090AB
:1030F600F7EAF0A3F0439A02221244B485822885A7
:1031060028F005F07401800225E0D5F0FBF529E5ED
:103116002875F008A42419F52674F835F0F52790DB
:10312600FC657402F0022FDBD29022C29022AFF02F
:10313600AE83E58290F7F6F0EEA3F0EFA3F090F7FA
:10314600DBE06034D2919003E8125028C2919003DC
:10315600E8125028D2919003E8125028C2919003A9
:10316600E8125028D2919003E8125028C291900399
:10317600E812502890FFFF2290F7F6E0FDA3E0FE4C
:10318600A3E0FF90F7CCEDF0EEA3F0EFA3F090F7FD
:10319600CFE537F0E538A3F090F7DB7401F0900047
:1031A6000022AF83E58290F7F9F0EFA3F090F7DB0A
:1031B600E06034D2919003E8125028C2919003E85F
:1031C600125028D2919003E8125028C2919003E839
:1031D600125028D2919003E8125028C2919003E829
:1031E60012502890FFFF2290F7F9E0FEA3E0FF7D42
:1031F6000090F7CCEEF0EFA3F0EDA3F090F7CFE55B
:1032060039F0E53AA3F090F7DB7401F09000002264
:103216007F0290DE0EE4F090F7CFE0FDA3E0FEC360
:1032260074409DE49E50047C4080048D047F0A8C8B
:10323600027B00EDC39AFDEE9BFE90F7CFEDF0EE1C
:10324600A3F08C06EE603690F7CCE0FBA3E0FCA37F
:10325600E0FD8B828C838DF012584990DE20F09031
:10326600F7CCE0FBA3E0FCA3E0FD0BBB00010C9058
:10327600F7CCEBF0ECA3F0EDA3F01E80C790DE11C7
:10328600E04FF090F7CFE0FEA3E0FF4E700590F719
:10329600DBE4F02290F7DB7402F07582002290F7EF
:1032A600D1E0FDA3E0FEA3E0FF90DE11E0FCB40157
:1032B60000E433FC20E0F290DE0EE4F090DE16E04F
:1032C600FC7B0090F7D4ECF0EBA3F090F7DAE0FC8F
:1032D60030E11390F7DB7403F090DE11E0FC740428
:1032E6004CF090FFFF2290F7DAE04402F090F7D41A
:1032F600E0FBA3E0FCC374409BE49C501CD291907D
:10330600012CC007C006C005125028C29190012C9E
:10331600125028D005D006D00790F7D4E0FBA3E0E2
:10332600FC8D07EB4C601690DE20E0FD8F828E83CD
:10333600F0A3AF82AE831BBBFF011C80E6E52C45E4
:103346002D6009852C82852D8312148990F7D4E08F
:10335600FEA3E0FFC3EE9440EF9400501DE52A451E
:103366002B6009852A82852B8312148990DE11E051
:10337600FF74084FF090F7DBE4F090DE11E0FF7485
:10338600404FF090F7D4E0FEA3E08E82F5832285CD
:10339600822E85832F2285823085833122753701DF
:1033A60075380090002575F040023134AFF0AE83D9
:1033B600E58290F7FBF0EEA3F0EFA3F090F7FBE0C9
:1033C600FDA3E0FEA3E0FF74022DFDE43EFE8D8228
:1033D6008E838FF0125849FDA31258498D25752208
:1033E6000122AF827D957E5A8D828E83A3E090F76F
:1033F600FEF0AC1490F7FEE0FBBBFF02803EEBB59F
:103406000723EC700890F7FE74FFF080E71C8D82AE
:103416008E83E02DFDE43EFE8D828E83A3E0FB903D
:10342600F7FEF080CF8D828E83E02DFDE43EFE8D8B
:10343600828E83A3E0FB90F7FEF080B88D828E83A8
:1034460022AFF0AE83E58290F7FFF0EEA3F0EFA394
:10345600F090F7FFE0F53DA3E0F53EA3E0F53F74FD
:1034660002253DFAE4353EFBAC3F8A828B838CF025
:10347600125849F8A3125849F9893B753C00740261
:10348600B53B06E4B53C0280227407B53B06E4B5BD
:103496003C028002804274AF58FE7F008A828B8392
:1034A6008CF0EE1256B2A3EF1256B28A828B838C40
:1034B600F0125849FAA3125849F5828A141233E8D1
:1034C600AE82AF8390F802EEF0EFA3F08E828F8388
:1034D600A3A3E0FE7F00801C898288141233E8AC27
:1034E60082AD8390F802ECF0EDA3F08C828D83E040
:1034F600FCFE7F007406253DFBE4353EFCAD3F8BAC
:10350600828C838DF0125849FCA3125849FDC3ECF6
:103516009EED9F50048C068D07EE4F700990DE11CC
:10352600E0FD74204DF090F802E0FCA3E0FD8E393A
:103536008F3A8C828D830231A890DE0EE4F090DE05
:1035460011E0FF30E40E90F7DBE4F090DE11E0FED0
:1035560074804EF0EF30E22490DE11E4F090FC66C9
:103566007404F090F7DBE4F0D291900014C00712D7
:103576005028C291900014125028D00790F7DBE033
:10358600FEBE0319D291900032C007125028C29194
:10359600900032125028D00790F7DBE4F090F7DB6A
:1035A600E0600302387FEF20E00302387F90DE0EF2
:1035B600E4F090DE16E0FFFE7B407C007D40EE608E
:1035C6001690DE20E0FA8B828C838DF01256B2A321
:1035D600AB82AC831E80E7E540FE20E7030237524C
:1035E60074605EFD6015BD200302370CBD4003020A
:1035F6003718BD600302373D023867741F5EFF70DF
:1036060041AD41BD0002801CBD06028005BD0826F5
:10361600800C90004075F040123447023867123330
:10362600A3023867753702753800905A7375F080B3
:1036360012313402386790004075F0401243A102FF
:103646003867BF0145AD41BD00028005BD0A268031
:1036560012753702753800905A7375F0801231343E
:10366600023867753701753800905A7675F0801202
:10367600313402386790DE11E0FD74204DF0900081
:103686004075F0401243A1023867BF0236AD41BD16
:1036960000028008BD120302386780127537027572
:1036A6003800905A7375F08012313402386790DE14
:1036B60011E0FD74204DF090004075F0401243A1DA
:1036C600023867BF032BE4B541127537027538001F
:1036D600905A7375F08012313402386790DE11E02B
:1036E600FD74204DF090004075F0401243A1023861
:1036F6006790004075F0401243A190DE11E0FD7422
:10370600204DF002386790DE11E0FD74204DF00286
:103716003867E52E452F6013123723800BC02EC065
:103726002F90004075F0402202386790004075F0F7
:103736004012389602386790DE11E0FD74204DF095
:1037460090004075F0401243A102386774605EFD38
:103756006015BD200302381EBD4003023832BD602D
:1037660003023855023867741F5EFF7048AE41BECB
:103776000103023867BE0303023867BE0502800BE9
:10378600BE0703023867BE0917800990DE00E542CE
:10379600F002386790004075F0401233B202386785
:1037A60090004075F0401243A190DE11E0FE7420B7
:1037B6004EF0023867BF0129AE41BE0103023867E9
:1037C600BE0303023867BE110302386790004075D6
:1037D600F0401243A190DE11E0FE74204EF0023854
:1037E60067BF0220AF41BF01028076BF030280712E
:1037F60090004075F0401243A190DE11E0FF742066
:103806004FF0805D90DE11E0FF74204FF090004095
:1038160075F0401243A1804990004075F040124374
:10382600A190DE11E0FF74204FF08035E52E452F84
:10383600601212383D800BC02EC02F90004075F0EC
:103846004022801D90004075F040123896801290FC
:10385600DE11E0FF74204FF090004075F0401243F7
:10386600A190DE11E0FF74404FF0E5464547700930
:1038760090DE11E0FF74084FF090F7DBE0FFBF0128
:103886000312321690F7DBE0FFBF02030232A422D6
:10389600AFF0AE83E58290F804F0EEA3F0EFA3F06C
:1038A60090F804E0FDA3E0FEA3E0FF8D828E838FF7
:1038B600F0125849FC20E7030239F074012DFAE4AE
:1038C6003EFB8F048A828B838CF0125849FC601E63
:1038D600BC0102802BBC0202803CBC03028073BC8C
:1038E600040302398DBCFE030239AA023A56753723
:1038F6000275380090FC6575F000123134023A56B4
:1039060090DE00E0FC7B007539288B3A8C828B8335
:103916001231A8023A5674022DFAE43EFB8F048A4D
:10392600828B838CF0125849FAA3125849FB74060D
:103936002DF8E43EF98F04888289838CF012584969
:10394600F539A3125849F53A8A828B831231A802B7
:103956003A568D028E038F048A488B498C4A740628
:103966002DF8E43EF98F04888289838CF012584939
:10397600F537A3125849F538854882854983854A23
:10398600F0123134023A5690F7D1E0FAA3E0FBA3E5
:10399600E0FC753910753A008A828B838CF01231FF
:1039A600A8023A5674022DFAE43EFB8F0490FC6B93
:1039B6007478F0745AA3F07480A3F0751404751526
:1039C600008A828B838CF01250F4E5828583F04561
:1039D600F06012D29190012C125028C29190012CC5
:1039E600125028806B75C983806690F7F1E0FCBCA5
:1039F600015674022DFDE43EFE8D828E838FF012F9
:103A06005849FDA3125849FE90DE0EE4F090DE16EA
:103A1600E0FF7C007513088F828C83C007C006C048
:103A260005C004125074D004D005D006D007EF4C60
:103A3600601690DE20E0FB8D828E83F0A3AD82AE11
:103A4600831FBFFF011C80E690F7DAE054FDFFF00C
:103A56009000002290F7ECE0FF30E10A90FC6674DB
:103A660005F090FFFF2290DE0E7405F090DE16E062
:103A7600FF8F4B754C0090DE17E0FCE4254BF54BB1
:103A8600EC354CF54C90F7EAE0FCA3E0FD4C7058A1
:103A960090F7E6E4F0A3F090DE2AE090F7E8F090E5
:103AA600DE2AE090F7E9F090DE2AE0FD7C0090F750
:103AB600EAEDF0ECA3F090DE2AE0FAE4FB2DFDEA55
:103AC6003CFC90F7EAEDF0ECA3F0E54B24FCF54B5B
:103AD600E54C34FFF54CC374049D74029C50099068
:103AE600F7EA7404F003A3F0E52955D16012D291E8
:103AF600900014125028C29190001412502880E8A9
:103B060090F7E3E0FBA3E0FCA3E090F7E6E0FAA37E
:103B1600E0FFEA2BFBEF3CFC7480252942D6852684
:103B26008285278374DEF0852682852783A3742AFF
:103B3600F0852682852783A3A38C07EFF08526824E
:103B4600852783A3A3A3EBF0852682852783A3A3DA
:103B5600A3A3A3A3A3E0543FF0852682852783A3CE
:103B6600A3A3A3A3A3A3E054CF4410F07405252672
:103B7600FEE43527FF90DE16E0FD8E828F83EDF0A2
:103B860074042526FEE43527FF90DE17E08E828F2B
:103B960083541FF5F0E054E045F0F090F7E6E0FEC0
:103BA600A3E0FFEE254BFCEF354CFDC374049C747B
:103BB600029D500B7404C39EF54B74029FF54CC3D3
:103BC6007440954BE4954C502890FC667406F09032
:103BD600DE14E0FD74FE5DF07513049000051250CE
:103BE60074751310854B82854C8312507490FFFEBA
:103BF60022E52942D6E52942D7E54B2EFEE54C3F84
:103C0600FF90F7E6EEF0EFA3F0E52955D160FAE56F
:103C160029F452D190F7E6E0FEA3E0FF90F7EAE040
:103C2600FCA3E0FDC3EE9CEF9D402C90F7ECE04436
:103C360002F090F7EAE4F0A3F090DE0E7405F0AE21
:103C46002374BF5524FF8E238F2490DE14E0FF7467
:103C5600FE5FF09000012290DE0E7405F0AE237434
:103C6600BF5524FF8E238F2490DE14E0FF74FE5F81
:103C7600F09000002290F7ECE0FF20E1012290F79F
:103C8600E3E0FDA3E0FEA3E0FF90F807EDF0EEA36E
:103C9600F090F7E8E0F55474FFB554028003024152
:103CA6000D90F7E9E0FBBB800050030240EFEB24E8
:103CB6006F50030240EFEB2480FA240A83F582EA70
:103CC600241583F583E473EF841A57376E8FA6DFC6
:103CD600C8EFEFEFEF477AD63C3D3F3F3E3F3F3FD1
:103CE6003F3F404040404040408D828E838FF012DF
:103CF6005849FA74012DF54FE43EF5508A52755332
:103D06000090F7EAE552F0E553A3F0854F8285501F
:103D160083E0F5517401254FF554E43550F555A966
:103D2600518902E4F92552F552EA3553F55390F7D5
:103D3600EAE552F0E553A3F0855482855583E0F811
:103D4600854F82855083A3A3884D894EE0FAE425EA
:103D56004DF54DEA354EF54E854D35854E3690F787
:103D6600E8E0FA90F7E9E0F5328552338553348A74
:103D760082122E8690F7EAE4F0A3F00241058D82C6
:103D86008E838FF0125849FA8D828E83A38A4D75E1
:103D96004E00E0FA74022DF554E43EF5558A018989
:103DA60002E4254DF54DEA354EF54EA84DAA4E9046
:103DB600F7EEE8F0EAA3F090F7E6E0F9A3E0FAE917
:103DC60024FEF54DEA34FFF54E854D52854E53E5FA
:103DD600524553603D90F7EEE0F54FA3E0F5507481
:103DE60001254FF9E43550FA90F7EEE9F0EAA3F031
:103DF600855482855583E0FAA3858254858355854B
:103E06004F82855083EAF0155274FFB5520215535E
:103E160080BD90F7E8E0FA90F7E9E0F5327535EA0B
:103E26007536F77533027534008A82122E86024182
:103E36000590F7ECE0FA20E23C8D828E838FF0123B
:103E46005849FA8D828E83A38A4D754E00E0FA900A
:103E5600F80774022DF0E43EA3F08A018902E4F922
:103E6600254DF54DEA354EF54EA84DAA4E90F7EE86
:103E7600E8F0EAA3F090F7EAE0F9A3E0FA894D8AC0
:103E86004EC37440954DE4954E5006754D40754EA3
:103E960000E9C3954DF9EA954EFA90F7EAE9F0EA9A
:103EA600A3F090F807E0F552A3E0F553854D54854D
:103EB6004E55E5544555603D90F7EEE0F54FA3E0CD
:103EC600F5507401254FF9E43550FA90F7EEE9F014
:103ED600EAA3F0855282855383E0FAA38582528550
:103EE6008353854F82855083EAF0155474FFB55489
:103EF60002155580BD90F7E8E0FA90F7E9E0F53253
:103F06007535EA7536F77533027534008A82122ED6
:103F160086024105D291900002C007C006C0051274
:103F26005028C291900002125028D005D006D00722
:103F360090F7E8E0FA90F7E9E0F53290F7E6E0F579
:103F460033A3E0F5348D358E368A82122E860241F1
:103F56000575357D75365A8B3275330D753400858A
:103F66005482122E8602410590FC67E0F8A3E0F920
:103F7600A3E0A3E0883589368B32753304753400A7
:103F8600855482122E8602410575356075365A8B28
:103F960032753313753400855482122E860241051C
:103FA60090F7E6E0F533A3E0F5348B328D358E36A7
:103FB600855482122E869000C81250281244D402CC
:103FC600410575355775365A8B3275330975340088
:103FD600855482122E860241058D828E838FF012C1
:103FE6005849FC74012DF9E43EFABC0202800ABC71
:103FF60003028021BC0429800DC002C00112459D28
:10400600D001D002801AC291C002C0011245FDD073
:1040160001D002800BC002C0011245BED001D00201
:1040260090F7E8E0FC90F7E9E0F53290F7E6E0F586
:1040360033A3E0F53489358A368C82122E86024106
:104046000590F7EA7401F0E4A3F07535367536DFAE
:1040560090F7E8E0FC90F7E9E0F53290F7EAE0F552
:1040660033A3E0F5348C82122E8690F7EAE4F0A3AF
:10407600F00241058D028E048C017C0090FC6B746D
:104086008BF0745AA3F07480A3F07514098C158A0A
:104096008289838CF0C007C006C0051250F4E58201
:1040A6008583F0D005D006D00745F0705275C980DB
:1040B60090F7E8E0FC90F7E9E0F53290F7E6E0F5F6
:1040C60033A3E0F5348D358E368C82122E86802F02
:1040D60090FC65E4F090FC66F090F809EDF0EEA334
:1040E600F0758202124135801690F7E6E0F533A3AB
:1040F600E0F5348B328D358E36855482122E8690BD
:10410600F7ECE054FDF022E5304531601985308248
:10411600853183121489AE82AF83EE4F701090F70B
:10412600ECE054FDF02290F7ECE054FDFFF022E5C0
:104136008290F80BF090F7ECE054FDF090F7E8E091
:10414600FF90F7E9E0F53290F80BE0FE8E33753418
:104156000090F809E0F535A3E0F5368F82022E8649
:10416600E52330E01175220274FE5523FEAF248E3E
:10417600238F2443BE01E5235406602F90FC65740B
:104186000AF075220374FD5523FEAF248E238F2477
:1041960090DE01E0FF74044FF09000081250289062
:1041A600DE01E0FF74FB5FF075220190DE0EE4F0A5
:1041B60090DE11E0FF30E21A90DE11E0FF74DB5F63
:1041C600F090F7CFE4F0A3F090F7D4F0A3F090F7D7
:1041D600DBF090DE0E7405F090DE11E0FF30E52096
:1041E60090DE11E0FF74CF5FF090FC667408F090EB
:1041F600F7E1E4F0A3F090F7E6F0A3F090F7EDF026
:1042060090DE14E0FF30E62090DE14E0FF749F5F3E
:10421600F090FC667408F090F7E1E4F0A3F090F7F4
:10422600E6F0A3F090F7EDF0E52320E2057404B57F
:104236002214122FDB90FC65740BF074FB5523FEE1
:10424600AF248E238F24E52330E41112353F74E723
:104256005523FE740F5524FF8E238F24E52430E664
:104266005490FC65740CF0123A5AAE82AF83BEFECF
:1042760041BFFF3E90F80C7406F0E4A3F090F7E817
:10428600E0FF90F7E9E0F53275350C7536F87533D1
:10429600027534008F82122E8690F7E8E0FF75359E
:1042A6000C7536F87532017533027534008F82123B
:1042B6002E86123C7BE52354E07006E52454BD604F
:1042C6002990FC667409F075130890004412507426
:1042D600852382852483751310125074741F552309
:1042E600FE74425524FF8E238F2422C0E0C082C074
:1042F60083C007C006C005C004C0D075D000E5BEA7
:1043060030E6FB90DE06E0FF7E00E5234207E5246B
:1043160042068F238E2490DE02E0FDE4CDC4CD6DEF
:10432600CD54F0CD6DFCED4207EC42068F238E2472
:1043360090DE04E025E0FCE4FD4207EC42068F2314
:10434600EEF52430E11290F7ECE054FEF0AE237463
:10435600FD5524FF8E238F24758B00C2E8D0D0D064
:1043660004D005D006D007D083D082D0E032C0E09A
:10437600C007C0D075D000E5BE30E6FBC2AFE58908
:1043860030E703752203AFBE74FC5FF5BE75890086
:0C439600C2C5D2AFD0D0D007D0E0322298
:105A570053444343763335300059415244535449F4
:105A6700434B4F4E45207230343530000000000064
:105A7700005253544E00554E494D504C454D454EDE
:105A87005445440052455345545F4E4F5700120149
:105A9700100100000040501D5B600001010203017E
:105AA7000A06100100000040010009022000010160
:105AB7000080FA09040000020000010007058502C2
:105AC70040000107050502400001040309042803FB
:105AD70047007200650061007400200053006300F6
:105AE7006F007400740020004700610064006700C5
:105AF7006500740073001E03590041005200440002
:105B0700200053007400690063006B0020004F0001
:105B17006E0065000A03300030003900330000FFD3
:1043A200AF83E58290F80EF0EFA3F090F80EE0FEF6
:1043B200A3E0FF7C007D008E028F038A828B83E064
:1043C200F9A3AA82AB83E960070CBC00EE0D80EB77
:1043D2007532F08C338D348E358F367582FE022E17
:1043E20086AF83E58290F810F0EFA3F090F810E02A
:1043F200FEA3E0FF7C007D008E028F038A828B8306
:10440200E493F9A3AA82AB83E960070CBC00ED0D2B
:1044120080EA8E358F367532F08C338D347582FE9C
:10442200022E86E58290F812F07535127536F8750F
:1044320032F17533017534007582FE022E86AF8328
:10444200E58290F813F0EFA3F07535137536F87521
:1044520032F27533027534007582FE022E86AF8207
:10446200AE83ADF0FC90F815EFF0EEA3F0EDA3F003
:10447200ECA3F07535157536F87532F3753304759E
:0844820034007582FE022E8653
:0514E400E4F50DF50E1A
:10448A007E197FF88FD57E197FF88ED47E217FF82A
:10449A008FD37E217FF87F008ED28F147515188FE7
:1044AA001690F81975F0000255F27403B50D06E47A
:1044BA00B50E02800280047582FF22AE0DAF0E0592
:1044CA000DE4B50D02050E8E822290DF46E0FFBF95
:1044DA00F00E90DF47E0FFBF0D0690DF487469F0E9
:1044EA00C2AF759A0075B80075A800123131AFBE17
:1044FA00747F5FF5BE75D69FC291020000221256E4
:10450A0066AC82AD83AEF0FFC004C005C006C0072A
:10451A009037BD75F086743D1254EEAC82AD83AE11
:10452A00F0FFE58124FCF581E4C0E0C0E074C0C07E
:10453A00E07441C0E08C828D838EF0EF125786AC16
:10454A0082AD83AEF0FFE58124FCF5818C828D83F8
:10455A008EF0EF125679AC82AD83AEF090DF09EEA1
:10456A00F08D0390DF0AEBF090DF0BECF02275E19F
:10457A000490DF3BE0FFBF01F890FC3CE0F5E190DE
:10458A00FC3CE0FFBF04012290DF3BE0FFBF0102D9
:10459A0080ED2290FC3CE0FFBF02012290DF13E095
:1045AA00FF74F05FF0E0FF740F4FF090FC3C740270
:1045BA00F0024A1290FC3CE0FFBF03012290DF1395
:1045CA00E0FF74F05FF0E0FF740A4FF090FC3C7477
:1045DA0003F090FCACE024FF92A0C2A490FCACE0F3
:1045EA006401FF24FF92A375E10390DF3BE0FFBF64
:1045FA0013F82290FC3CE0FFBF04012290DF13E095
:10460A00FF74F05FF0AF9174EF5FF591C2A0C2A49E
:10461A00D2A375E10490DF3BE0FFBF01F8AF9B74C2
:10462A00FC5FF59BAFE974EF5FF5E990FC3C74041D
:10463A00F02290FC3FE4F0A3F090FC32F0A3F0905B
:10464A00FC34F0A3F053C6C7759D00859E9E439E19
:10465A000485A9A943B90190FC3C7404F0751400BF
:10466A00751500F51690F83275F0001255F2122DF4
:10467A0036D2A87591D175E900750F00439A01C227
:10468A00A0C2A4D2A375E10490DF3BE0FFBF01F80A
:10469A00227E007F00C3EE94DCEF9405502490DF65
:1046AA003CE0FD5450600490000122900032C007A3
:1046BA00C006125056D006D00774322EFEE43FFFD1
:1046CA0080D390000022AF83E58290FC5CF0EFA3D8
:1046DA00F090FC5EE4F090DF02E0FF90DF3BE0FE4A
:1046EA00BE130BB291C007124166D00780EDC2918A
:1046FA0090FCAAE4F090FC58E0FDA3E0FE90FCA038
:10470A00EDF0EEA3F090FC5AE0FBA3E0FC90FCA6CF
:10471A00EBF0ECA3F090FC56E0F9A3E0FA90FCA2CF
:10472A00E9F0EAA3F090FCA4E9C39BF0EA9CA3F0A9
:10473A0090FCA4E0FBA3E0FC8D148E158B828C8385
:10474A00C007C006C005C002C0011256CDAB82AC7C
:10475A0083D001D002D005D006D00790FCA8EB295F
:10476A00F0EC3AA3F0E94A705D90FC5CE0FBA3E050
:10477A00FC8B828C83E0F8881075110090FC56E55A
:10478A0010F0E511A3F090DF04E0F8530003B8003D
:10479A00028018B80102800302486290FC56740134
:1047AA002510F0E43511A3F002486290FC5C740114
:1047BA002BF0E43CA3F090FC56E0FBA3E0FC90DF76
:1047CA0002EBF002486290DF04E0FC530403BC00F1
:1047DA00028046BC0102800302486290FC5CE0FB56
:1047EA00A3E0FC90FC5FE9F0EAA3F090FC6174019D
:1047FA00F0E4A3F08B828C83C007C002C001124F81
:10480A00D3D001D002D00790FC5CE0FBA3E0FC8986
:10481A00008B828C83E8F0803FED4E603690FCA8D6
:10482A00E0FDA3E090DF02EDF090DF04E0FE74FC0F
:10483A005EF090FCA8E0FDA3E0FEC374FF9DE49E39
:10484A00500990DF04E0FE74024EF090FCAA740155
:10485A00F0800590DF02E9F0D2A890FCABE0FE20E0
:10486A00E30302499090DF04E0FE530603BE01060B
:10487A0090FC5E7401F090FC5EE0FE90FC5CE0FC53
:10488A00A3E0FDEE2CFAE43DFB90FC56E0F8A3E031
:10489A00F990FC7DE8F0E9A3F08A828B83C007C017
:1048AA0006C005C00412532FAA82AB83D004D005D8
:1048BA00D006D00790FCABE0F9530104B90448C014
:1048CA0007EE2CF8E43DF990FCABE0FF5307F090BB
:1048DA00FC81E8F0E9A3F090FC83EAF0EBA3F09006
:1048EA00FC85EFF088828983C007C006C005C00432
:1048FA00C003C002125369D002D003D004D005D03D
:10490A0006D007D0078046C007EE2CF8E43DF990A0
:10491A00FCABE0FF5307F090FC88E8F0E9A3F090C5
:10492A00FC8AEAF0EBA3F090FC8CEFF08882898392
:10493A00C007C006C005C004C003C0021253B2D0EB
:10494A0002D003D004D005D006D007D007EE601EEF
:10495A0090FCABE0FE5306F0BE50098C828D837446
:10496A0010F080228A068C828D83EEF0801890FCEB
:10497A00ABE0FE5306F0BE500890DF027410F080E0
:10498A000590DF02EAF090FC5CE0FDA3E0FE90FCFB
:10499A0038EDF0EEA3F090FC9EE4F0A3F090FCACAE
:1049AA00E024FF92A0C2A490FCACE0640124FF9230
:1049BA00A375E1037D607EEA90DF3BE0FCBC130255
:1049CA00801C1DBDFF011EED4E6013B291C007C0D1
:1049DA0006C005124166D005D006D00780DAD2910A
:1049EA00ED4E700690FC667413F090DF3BE0FEBE5D
:1049FA00130BB291C007124166D00780EDC29190A5
:104A0A00DF02EFF075820122D2A875140075150035
:104A1A0075160290F83275F0001255F290FC32E4E5
:104A2A00F0A3F090FC34F0A3F090FC36F090FC3741
:104A3A0004F090F831E4F0AF9B74FC5FF59BAFE9AA
:104A4A0074EF5FF5E9C2A090FCACE024FF92A4E009
:104A5A006401FF24FF92A375E10290DF3BE0FFBFF0
:104A6A000DF84391102290FCAD7401F02290FCAD38
:104A7A00E4F022C021C0E0C0F0C082C083C007C0F9
:104A8A0006C005C004C003C002C001C000C0D07582
:104A9A00D00090FC657411F0C28990DF3BE0FFBF43
:104AAA000D028003024BC7D29190FC97E0E0602A86
:104ABA0090FC98E0FEA3E0FF90FC98E024FFFCA3A2
:104ACA00E034FFFD90FC98ECF0EDA3F074FF2F406A
:104ADA000990DF04E0FF74FC5FF090FC3C7402F084
:104AEA0090F831E025E0FEE42432FFEE34F8FEE0EF
:104AFA0075F002A42432FC74FC35F0FD8C828D839F
:104B0A00E0FAA3E0FB74012AF8E43BF98C828D8376
:104B1A00E8F0E9A3F0EA2FF582EB3EF583E5D9F058
:104B2A0090F831E075F002A42432F58274FC35F075
:104B3A00F583E0FEA3E0FFC39402501A90F831E037
:104B4A0075F002A42432F58274FC35F0F583E0FE98
:104B5A00A3E0FF4E701A90F831E0FF75F002A4242A
:104B6A0032F58274FC35F0F58374FFF07401A3F01A
:104B7A0090FC98E0A3E090FC98E0F5F0A3E045F003
:104B8A006003024D8490FC97E0E07003024D84902C
:104B9A00FC9AE0FEA3E0FF90FC98EEF0EFA3F09001
:104BAA00FC98E0FEA3E090DF02EEF090DF04E0FF65
:104BBA0074FC5FF0E0FF74024FF0024D8490DF3B1B
:104BCA00E0FFBF13028003024D8490FCAAE0E0706C
:104BDA0003024D1590FC4EE0FEA3E0FF0EBE00015D
:104BEA000F90FC4EEEF0EFA3F090FC9EE0FEA3E0E7
:104BFA00FF90FCA2E0FCA3E0FDEEB50406EFB505CC
:104C0A00028003024CE890FCA0E0A3E090FCA0E044
:104C1A00F5F0A3E045F0603790FCA0E0FEA3E0FFCA
:104C2A00BEFF05BF0002801490FCA0E024FFFEA393
:104C3A00E034FFFF90FCA0EEF0EFA3F090FCA6E0BA
:104C4A00FEA3E0FF90FC9EEEF0EFA3F0024CE8908A
:104C5A00FCA2E0F514A3E0F51590FC9CE0FF7E00B1
:104C6A008F828E831256CDAE82AF8390FC38E0FCE1
:104C7A00A3E0FDEE2CF582EF3DF583E4F090FC9C79
:104C8A00E02401F0E0FF90FC9DE0FEEFB506059000
:104C9A00FC9CE4F090FCA2E0F514A3E0F51590FC6E
:104CAA009CE0FF7E008F828E831256CDAE82AF8348
:104CBA0090FC38E0FCA3E0FDEE2CFEEF3DFF8E8277
:104CCA008F83E0701090FC41E4F090FC667412F05F
:104CDA00124578C29190FC9E7401F0E4A3F090FC16
:104CEA00A8E0FEA3E0FF90FCA8E024FFFCA3E034C8
:104CFA00FFFD90FCA8ECF0EDA3F0BEFF22BF001F61
:104D0A0090DF04E0FF74FC5FF0801490FCA8E024BC
:104D1A00FFFEA3E034FFFF90FCA8EEF0EFA3F090B3
:104D2A00FC3C7403F090FCA2E0F514A3E0F51590A6
:104D3A00FC9CE0FF7E008F828E831256CDAE82AF3E
:104D4A008390FC9EE0FCA3E0FD90FC9EE02401F031
:104D5A00A3E03400F0EC2EFEED3FFF90FC38E0FCBF
:104D6A00A3E0FDEE2CF582EF3DF583E0F5D990FC4A
:104D7A003AE02401F0A3E03400F0D0D0D000D00112
:104D8A00D002D003D004D005D006D007D083D08279
:104D9A00D0F0D0E0D02132C021C0E0C0F0C082C043
:104DAA0083C007C006C005C004C003C002C001C05A
:104DBA0000C0D075D00075120090FC657410F0AE7A
:104DCA009B74FC5EF59BE5E9420FE5E930E0209033
:104DDA00FC3DE0FDA3E08D067D00AB9C7C0090FCD1
:104DEA003FED4BF0EE4CA3F0AEE974FE5EF5E9E55B
:104DFA00E954707003024F8490FC3CE0FEBE030A43
:104E0A00AE0F748F5EF50F024F7D90F831E0FEB45D
:104E1A000100E4332436F582E434FCF583E0FEBE77
:104E2A0001028003024F5A90FCABE0FE20E103022C
:104E3A004F3390DF04E0FE530603BE0103751201EF
:104E4A0090FCABE0FE530601BE017090F831E025FC
:104E5A00E0FDE42432FEED34F8FDAB127C00EB2ECB
:104E6A00FEEC3DFDE0F929FAE42432F9EA34F8FAD5
:104E7A00EB29FBEC3AFCE075F002A42432F58274CB
:104E8A00FC35F0F583E0F9A3E0FAA8127F00E9C344
:104E9A0098F9EA9FFA90FCABE0FF5307F090FC8187
:104EAA00EBF0ECA3F090FC83E9F0EAA3F090FC8528
:104EBA00EFF08E828D83125369806E90F831E0256F
:104ECA00E0FEE42432FFEE34F8FEAC127D00EC2F53
:104EDA00FFED3EFEE025E0FAE42432FBEA34F8FA7C
:104EEA00EC2BFCED3AFDE075F002A42432F5827455
:104EFA00FC35F0F583E0FAA3E0FBA8127900EAC3D7
:104F0A0098FAEB99FB90FCABE0F95301F090FC881E
:104F1A00ECF0EDA3F090FC8AEAF0EBA3F090FC8CA5
:104F2A00E9F08F828E831253B290F831E0FF740158
:104F3A006FF0E0FF75F002A42432F58274FC35F0BC
:104F4A00F583E4F0A3F090FC36F090FC37F0802172
:104F5A0090FC667412F0B29190F831E0FF75F0029D
:104F6A00A42432F58274FC35F0F583E4F0A3F0B2A0
:104F7A0091C291AFE974CF5FF5E9E5E930E61490A3
:104F8A00FC667410F0B291124578B291AFE974BF21
:104F9A005FF5E9E5E930E71490FC667411F0B29127
:104FAA00124578B291AFE9747F5FF5E9D0D0D000AD
:104FBA00D001D002D003D004D005D006D007D083C8
:104FCA00D082D0F0D0E0D02132AF83E58290FC636A
:104FDA00F0EFA3F090FC61E0FEA3E0FF90FC63E039
:104FEA00FCA3E0FD90FC5FE0FAA3E0FB8A008B01E2
:104FFA001ABAFF011BE8496024EE2AF8EF3BF9E8E8
:10500A002CF8E93DF9EA2CF582EB3DF583C006C0A0
:0E501A0007E088828983F0D007D00680CF227D
:105B2700000000000000010000000000000000006D
:075B37000000000000000067
:10502800AE82AF831EBEFF011FC3E49E74808FF063
:1050380063F08095F050167C4C7D04EC24FFFAED6B
:1050480034FFFB8A048B05EA4B70F080D722AE82CE
:10505800E583CE25E0CE33FF1EBEFF011FC3E49ECD
:1050680074808FF063F08095F040ED22AE82AF83BC
:10507800D2919003E8C007C006125028C29190014F
:10508800F4125028D006D0071513AD13ED20E754BD
:10509800EE30E024900019C007C006C00512502861
:1050A800D291900226125028C291900019125028CD
:1050B800D005D006D0078022900113C007C006C0D3
:1050C80005125028D291900032125028C2919001B6
:1050D80013125028D005D006D007EFC313CE13CE35
:1050E800FF1D80A8C2919003E8025028AFF0AE835C
:1050F800E58290FC6EF0EEA3F0EFA3F090FC6EE07A
:10510800FDA3E0FEA3E0FF90FC6BE0FAA3E0FBA3A5
:10511800E0FCA814A915E8496050C000C0018D82C0
:105128008E838FF0125849F98A828B838CF012583B
:1051380049F8E9C398F98916D001D0006010E5163E
:10514800F5173395E0F518851782851883220DBD6C
:1051580000010E90FC6EEDF0EEA3F0EFA3F00ABA9A
:1051680000010B18B8FF011980AC90000022AFBEF7
:1051780074FB5FF5BEE5BE30E6FBAFC674B85FF5FD
:10518800C6E5C620E6FB43BE04E5BE30E6FB53C6D3
:10519800C743E40C43E401D2B92243FE0F43FF198D
:1051A800C292C293C2A0C2A4D2A3C29122C0E0C03C
:1051B80082C083C0D090FC67E02401F0A3E03400F3
:1051C800F0A3E03400F0A3E03400F0D0D0D083D0D6
:1051D80082D0E0321244B4AF8290FC75EFF08FF0C9
:1051E80005F07401800225E0D5F0FB90FC76F0EF25
:1051F80075F008A42419FE74F835F0FF90FC71EEE0
:10520800F0EFA3F08E828F83A3A374DFF08E828FDA
:1052180083A3A3A374B1F08E828F83A3A3A3A3A3B4
:105228007410F074062EF582E43FF583E054E044F0
:105238001DF074072EF582E43FF583E0543F4440A7
:10524800F074072EF582E43FF583E054FC4401F046
:105258001244B4AF8290FC77EFF08FF005F0740140
:10526800800225E0D5F0FB90FC78F0EF75F008A4FB
:105278002419FE74F835F0FF90FC73EEF0EFA3F0FC
:105288008E828F8374DFF08E828F83A374B2F08E48
:10529800828F83A3A3A3A3A37410F074062EF582B0
:1052A800E43FF583E054E0441EF074072EF582E4F1
:1052B8003FF583E054CF4410F074072EF582E43FA5
:1052C800F583E054FC4401F043A91043B91022AF20
:1052D80083E58290FC7BF0EFA3F0E5B330E3FB902D
:1052E800FC71E0FEA3E0FF90FC7BE0FCA3E0FD8CFA
:1052F800028D038B028E828F83EAF090FC71E0FEB0
:10530800A3E0FF8E828F83A37D00ECF090FC76E013
:1053180042D690FC79E0FF90FC7AE0FE4F4401F51C
:10532800B3E5B330E3FB22AF83E58290FC7FF0EF77
:10533800A3F090FC7FE0FEA3E0FF90FC7DE0FCA3DF
:10534800E0FDEC540F60158C028D030CBC00010DC0
:10535800EA2EF582EB3FF583E4F080E68C828D83BC
:1053680022AF83E58290FC86F0EFA3F090FC86E004
:10537800FEA3E0FF90FC81E0FCA3E0FD90FC83E04D
:10538800FAA3E0FB90FC85E0F990FC8FECF0EDA32C
:10539800F090FC91EAF0EBA3F090FC93E4F090FC21
:1053A80094E9F08E828F830253FCAF83E58290FCF0
:1053B8008DF0EFA3F090FC8DE0FEA3E0FF90FC8859
:1053C800E0FCA3E0FD90FC8AE0FAA3E0FB90FC8CF3
:1053D800E0F990FC8FECF0EDA3F090FC91EAF0EB93
:1053E800A3F090FC937402F090FC94E9F08E828F05
:1053F800830253FCAF83E58290FC95F0EFA3F0E5C0
:10540800B330E3FB90FC95E0FEA3E0FF90FC8FE057
:10541800F51AA3E0F51B90FC94E0FB74505BF519BA
:1054280090FC93E0F94B4401FB740149F51890FC9A
:1054380091E0F514A3E0F515E4F516F517C3E516A4
:105448009514E5179515400122C00390FC71E0F80A
:10545800A3E0FBE5162EF9E5173FFA89048A058DC6
:105468000488828B83ECF090FC71E0FCA3E0FD8C57
:10547800828D83A3E9F090FC73E0FCA3E0FD8C82AD
:105488008D83A3A3E516251AFCE517351BFD8C02B1
:105498008D038B02EAF090FC73E0FAA3E0FB8A82AA
:1054A8008B83A3A3A3ECF090FC78E0FD90FC76E05E
:1054B800FC4D42D6D003E5196017E51424F0FCE54D
:1054C8001534FFFDECB51609EDB517058518B38041
:1054D800028BB3E5B330E3FB74102516F516E435FB
:1054E80017F517025445125591BC0003025758EF9F
:1054F80060FA30D502B2D1E583B4FF0302576EE5F6
:1055080082B4FF0302576E258340072482400B02B2
:105518005758248314500302576EF582EA8DF0A47D
:10552800A8F0EA8EF0A428F8E435F0F9EB8DF0A4A1
:1055380028E935F0F9E433CA8FF0A429F9EA35F0FF
:10554800FAEBF88EF0A429F9EA35F0FAE433FBEC2B
:105558008DF0A429F9EA35F0FAE43BFBE88FF0A4D2
:105568002AFAEB35F0FBE433CCFD8EF0A42AFAEBF3
:1055780035F0FBE43CFCED8FF0A42BFBEC35F0FCA4
:1055880020E7031255BF025737AA82AB83A2F7332D
:1055980092D1F5826002D2F7ACF0E58124F9F8E601
:1055A800FD08E6FE0886F008E6A2F73392D5F583F3
:0755B8006002D2F7AFF02200
:0614BA00E478FFF6D8FD06
:1055BF007804EC7011E58224F8500AF582E4C9CA28
:1055CF00CBFCD8EF22EC7820058220E713D582019F
:1055DF0022C3E933F9EA33FAEB33FBEC33FCD8EAB5
:1055EF00158222AC82AD83AE15AF16BE0004EF60FC
:1055FF000C1F0FE5141256B2A3DEFADFF88C828D62
:10560F008322AD82AE83AFF08D198E1A8F1B851456
:10561F001C85151D85161EA817A91888038904183F
:10562F00B8FF0119EB4C6025851C82851D83851EF3
:10563F00F0125849FCA385821C85831D8D828E83B1
:10564F008FF0EC1256B2A3AD82AE8380CE85198255
:07565F00851A83851BF02270
:101498007917E94400601B7A01905B277897759368
:1014A800FCE493F2A308B800020593D9F4DAF275C4
:0214B80093FFA0
:10566600FCABF0AA83A982749EC2D1F5821255BF03
:105676000257377F9E1256A030D103025758C3EF08
:105686009582500974FFF5F0F583F58222790012B0
:10569600586589828A838BF0EC22AA82AB83A2F7B3
:1056A6003392D1F5826002D2F7ACF02220F71130A6
:1056B600F6138883A88220F509F6A883758300224D
:1056C60080FEF280F5F022E5828514F0A4C582C042
:1056D600F08515F0A4D0F025F0C5838514F0A42537
:1056E60083F58322E514451560467A01E51425E025
:1056F600F514E515334012F515E5829514E5839505
:105706001540030A80E6C3E51513F515E51413F5F0
:1057160014C3E5829514F5F0E58395154005F583E8
:1057260085F082C3E51513F515E51413F514DAE1D2
:015736002250
:1014C0007800E84400600A79007593F0E4F309D8E5
:1014D000FC7897E8440C600C790D90F000E4F0A3E0
:0414E000D8FCD9FA61
:02148900E4730A
:10573700B98003EA13B34010EA2401FAE43BFBE41F
:105747003CFC50047C800582BC000EBB000BBA00F9
:1057570008E4F5F0F583F58222A2D1E582138CF0F7
:1057670092F78B838A8222E4F583F58275F080F4C1
:10577700A2D11322E4F583F58275F0C0747F22125B
:10578700559130D502B2D1BF0009BC000302577B47
:1057970002576EBC0003025758E583B4FF0BE5823E
:1057A700B4FF0302577B025758E582B4FF03025741
:1057B7006EC395835007247F400B025758248014EB
:1057C700500302576EF582C3ED9AEE9BEF9C401192
:1057D7001582C3EA33F9EB33FAEC33FBE433FC808D
:1057E70005E4CCCBCAF9C08275F019C3E99DEA9EDE
:1057F700EB9FEC9400D5F002802D400EE99DF9EA6D
:105807009EFAEB9FFBEC9400FCC3B3E833F8E58208
:1058170033F582E58333F583C3E933F9EA33FAEBEA
:1058270033FBEC33FC80C4B3E4F938FAE43582FB8C
:10583700E43583FCD082500405827C801255BF0278
:02584700574FB9
:0D148B007581551258A8E582600302148691
:1058490020F71430F6148883A88220F507E6A88388
:1058590075830022E280F7E49322E0226040F82574
:1058690082500274FFF582E824F8501ECCCBCAF9A5
:10587900E4CC24F85014CBCAF9E4CB24F8500BCA71
:10588900F9E4CA24F8500379002224086010F8C307
:10589900EC13FCEB13FBEA13FAE913F9D8F12275BF
:0358A90082002258
:00000001FF
